:100000008CC0B3C0BEC3B1C0B0C0B4C0AEC0ADC080
:10001000ACC0ABC0AAC0A9C05DC1A7C0A6C0814585
:1000200086468B479048944997609B619E62A16386
:10003000A464A765AA66AC67AE68B069B280B481F3
:10004000B682B883BA84BB84BD84FF21000000005F
:100050000000000000000000000023456C98C9FF6C
:10006000040714233764A0FFFFFFFFFFFFFFFFFF1C
:10007000FFFFFF00000000000000000023405F7A47
:10008000B4FFFFFFFFFFFF001400081400080E1468
:100090000004080E14000305080E140004080A0EDC
:1000A0001114000305080A0E1014000305080A0EB7
:1000B0001012140008000E00080E0004080E0003C1
:1000C00005080E0004080E1100080E1100F3F404D8
:1000D000080E10121400080A0C0E0F10121400085B
:1000E0000EED14000203040500041400040E1400B5
:1000F000040810140004080F1114000305080A0E68
:100100000004080A0E00EEEDECEB140E08040004E7
:10011000080E00EBECEDEEF3F41411241FBECFE556
:10012000D1E0DEBFCDBF20E0A0E6B0E001C01D926F
:10013000AB37B207E1F7ECE7F0E085E5808781E0D7
:100140008383148212828683118211868BE08287D8
:1001500088E58387E1E6F0E08DEF87838EEF858386
:10016000712C55245A94B7D027C34ACF1BBC19BC55
:1001700018BC0895189525B7277E25BF29B722609A
:1001800029BF21E022BF019728F020E18895215066
:10019000E9F7F9CF089588EE93E0EDCF369A3699D6
:1001A000FECF95B18091600089270895CF93C72D28
:1001B00081E0870D8F73782E662D90E0EFD26FEF80
:1001C0008C2F90E0CF91EAC2FF920F931F93CF93B1
:1001D000DF93F82E0DE710E0CEE7D0E0F11005C078
:1001E000CE01D4D2F801808304C0F8016081CE0131
:1001F000D5D221970F5F1F4FC337D10579F7DF9114
:10020000CF911F910F91FF900895D0DF81E0DCCF57
:10021000811101C0ABCF815090E0FC01E45BFF4F46
:10022000E491EBBDFC01E05AFF4FE491E9BDFC0114
:10023000EC58FF4F849188BD08950F931F93CF937F
:10024000C82F8B01CC2359F085E0E2DFC80193DF92
:100250008DDFC80190DFC8018EDFC150F3CFCF9191
:100260001F910F910895EF92FF920F931F93CF93D9
:10027000C8E0E82EF12C062F10E084E1C9DFC701A9
:100280007ADF74DFC80177DFC150B9F7CF911F91D2
:100290000F91FF90EF9008951F93CF93DF938FEA14
:1002A00087B986EC86B91092600010E1C0E0D0E01A
:1002B00085E090E060DF72DFC80FD11D1150C1F7FB
:1002C000CE0124E0969587952A95E1F7DF91CF91AD
:1002D0001F910895189510927B0087E790E056D201
:1002E000853519F0612C91DF11C0712C872D90E0BC
:1002F0004DD2682E8F3F19F080E066DF07C0872D52
:1003000091E0970D792E803488F3F6CF80918500A7
:100310008111AB9820918600C0917F0010918000E0
:1003200080917D00882319F010E0C0E02AE12F5F62
:1003300090E040E050E0A8E8B0E0222379F0BD0171
:100340006F5F7F4FFB013197E491EE2319F0962FF9
:100350009A1BF6CF2150AD01DB01EFCF092F6C2F97
:1003600070E0A92FB0E0E02FF0E0112321F09D0113
:100370002E1B3F0B05C09F0121503109260F371F4F
:100380003197E40FF51FF49025593F4FF901F082A2
:10039000015049F79C0F90938800CC2371F01123F2
:1003A00029F0292F30E02150310902C020E030E04F
:1003B000F901E559FF4F41E0408327E0290F322F33
:1003C0003150E32FE91BF0E0ED5EFE4FE491A32FE7
:1003D000B0E0A559BF4FEC933913F2CFE22FF0E014
:1003E000E659FF4F31E050916B004081541330E0EB
:1003F000231B20938900362D353FE8F5452D4330EA
:10040000B0F480918A008F3F29F480917B00809323
:100410008A0006C081E0860D682E891708F0612CDD
:1004200080918A008F5F8F7180938A0024C0309101
:100430007B0030938A004730C0F430918200332330
:1004400011F0882339F081E0860D682E891798F025
:10045000612C11C0862D6916D9F3662019F08150E0
:10046000682E09C02150622E06C08111F1CF809103
:100470007E00882369F3512C8FEF8DBD80E68CBD03
:10048000AB9AAA9A8FE384BB83E187BB88EE88BBD3
:1004900081E083BF91EA9ABD80BF8BB780628BBF3A
:1004A0008AB785608ABF85B7806285BF78948CE201
:1004B00087B986EC86B93699FECF8FEF80936000BE
:1004C000C62DC53F10F0612C3CC080918A00803160
:1004D00038F4E62DF0E0E559FF4FC081DC2F31C044
:1004E0005ADE80917B0080938A00CDE7D0E000E067
:1004F00010E0FF24F39481E0800F0F5F1F4F98817D
:100500009F3F29F4219609301105A9F7E2CF6DE547
:1005100070E093DEF801EF59FF4F608088818F25EE
:10052000888373DE6FE070E080E287DE88818F254C
:100530008883612C6ADE2FDE80917D00882311F391
:10054000C8CF34DE10E0F12C8CE2D82E96ECC92E08
:10055000EE24EA94CE3E19F463E481E204C0CD3E79
:1005600021F468E284E17FDE76C0CC3E11F469E2DA
:1005700003C0CB3E19F462E581E0F5CFC33F81F4BF
:1005800004E084E145DE85E090E0F5DD88E040DED2
:1005900081E490E0F0DD0150A1F780ED92E05AC0D7
:1005A000C43F51F584E690E0E6DDF8DD90E0292FC8
:1005B00030E0F901E25EFF4FE491E81710F49E5F2E
:1005C000F6CFF901E15EFF4F04916DE770E0802FF7
:1005D00082958695877031DE8EEE92E0CCDD65E007
:1005E00070E081E02ADE85E694E0C5DD6DE770E02D
:1005F000802F8F7122DE0DC0CE3F71F400E000939A
:10060000860003DE6AEF70E081E017DE0F5F0A31DB
:10061000B1F7C1DDC0DD1FC0CD3F69F58FEF80931D
:100620008700F3DD85E0F4DDB6DDB5DD84E1F0DDE6
:1006300033DE80938700E9DDAEDDADDDF9CF36999D
:10064000FECFE0926000F394909187008917C8F480
:1006500084EF91E090DD80917B0080938A009EDDA5
:10066000803998F51F5F183008F474CFD53190F0B9
:1006700010E0DAE0CAE08D2FCBDD0EDED7B8C6B8C9
:10068000DECFDB3028F3F4E1FF1510F7E0927B00BA
:10069000DAE0DECFD23030F08D2F86958695D69574
:1006A000D80F12C063DD85B7877E806185BFF8945F
:1006B00085B7846885BF8B7F85BF85B7806285BF1E
:1006C000889585B78F7D85BFCD2F10E043CF11244E
:1006D00016B84CDD87B38C7E87BB20E041E034E068
:1006E00076B386B3883049F486B361E050E0843055
:1006F00009F460E0862F952F02C081E090E0999B7D
:1007000003C0511003C035C0009749F436E03515D9
:1007100090F5783081F121112EC040E039E0552D5F
:1007200061E0583008F060E0650F562E411105C0B9
:10073000211102C0282F01C021E0999885B7877E3A
:10074000806185BFA895832F887011F490E401C063
:1007500090E6832F8770892B81BD85B7846885BF1C
:100760008B7F85BF78948895F89481B58F7B81BD08
:10077000B7CF0097A1F68FE58DBF81E08EBF1FBE7A
:10078000AADD552011F0189501C0A1DFE199FECF37
:100790001FBA8EBBE09A99278DB30895262FE19951
:1007A000FECF1CBA1FBA8EBB2DBB0FB6F894E29ACF
:0C07B000E19A0FBE01960895F894FFCF67
